:020000040800F2
:10200000D0040020694900089D340008AB34000862
:1020100000000000000000000000000000000000C0
:10202000000000000000000000000000AF340008C5
:102030000000000000000000B13400089F340008D8
:10204000E32D00080000000083320008C3320008BE
:102050000F3900080F4900081B4900089149000882
:102060000000000093490008B322000895490008C9
:1020700097490008994900089B49000800000000A2
:102080009D4900089F49000800000000A149000880
:10209000A3490008A5490008A7490008A949000864
:1020A000AB490008AD490008AF490008B149000834
:1020B000B34900080121C206D20E9140CE4A1160F8
:1020C000704700B5BFF34F8FA148CC490860BFF3FC
:1020D0004F8F00BFFDE700B589B000209D49087013
:1020E000072000F05BFF002000F058FF00230122D2
:1020F0000B219020C00500F0FCFF002301220821E5
:102100009020C00500F0F5FF01220B219020C005B2
:1021100001F0A3F8012208219020C00501F09DF8EC
:10212000012000900323022209219020C00501F024
:1021300023F801200090032302220A219020C005E9
:1021400001F01AF8AE49AF4801F09CF8AD4801F033
:10215000B3F810200190002002908020039000200E
:10216000049000200590002006900020079001A90F
:10217000A54801F0A7F800200190002002908020DF
:1021800003900020049000200590002006908020FD
:102190008001079001A99D4801F094F801210A20CF
:1021A00001F0BFF80A20FFF785FF01210A2001F0A6
:1021B000B8F80A20FFF77EFFBB48007801210143F1
:1021C000B9480170B8480078DF210140B648017075
:1021D000B5480078FB210140B3480170B24800784F
:1021E000F7210140B048017009B000BD80B5AE488C
:1021F00000780100C907C90F00293DD0AA4800781E
:10220000C0B200090100C907C90F00293AD1022054
:1022100001F0F7F8002802D000204E4908704D4820
:102220000078012802D100F087FA2BE049480078B5
:10223000032802D100F00EFB24E046480078042871
:1022400002D100F089FB1DE042480078022802D14B
:1022500000F00AFA16E03F480078002802D100F0AA
:1022600029F90FE090480078202101438E48017041
:1022700000203849087005E08B4800782021014390
:102280008948017001BD88480078042101438648CF
:102290000170854800780821014383480170704728
:1022A000814800780100C9B249090800C007C00F81
:1022B000704780B57C480078C0B200090100C907AA
:1022C000C90F002927D079480068202108407749A4
:1022D0000860002812D0764800684006FBD54A48BE
:1022E00000680221884348490860D74800682021D7
:1022F0000143D548016000F08BF828E042480068AF
:102300000821884340490860CF4800688021014384
:10231000CD4801601BE03C480068082188433A49E9
:102320000860394800680221884337490860C64878
:102330000068802109010143C3480160C248006868
:10234000802189000143C048016000F061F801BDAF
:102350000400FA054008002038B50500524800780E
:10236000102101435048017001220B219020C0052B
:1023700000F073FF012208219020C00500F06DFFDE
:1023800000200400FF2C04D80020B0490855641C2C
:10239000F8E71D480068012188431B4908601B4875
:1023A00000680121884319490860A9480560A948C7
:1023B000A9490860A948AA49086013480068022191
:1023C00001431148016010480068082101430E488C
:1023D0000160A448006840210143A24801600A4806
:1023E00000680121014308480160CA480068802153
:1023F0000143C848016031BD00E100E00CED00E0A0
:1024000081060000003801401C00024030000240FC
:1024100010B525480078EF210140234801700022C3
:1024200008219020C00500F018FF00220B21902009
:10243000C00500F012FF00200400FF2C04D800208B
:1024400082490855641CF8E7B348006801218843B5
:10245000B1490860B148006801218843AF4908606C
:1024600080204000AE490860AE48AF490860774818
:10247000AE490860A948006802210143A7480160ED
:10248000A648006808210143A4480160A3480068E9
:1024900001210143A14801609E4800684021014399
:1024A0009C48016010BD0000E407002000000240CD
:1024B0001C380140F8B59E480078C0B240080100C1
:1024C000C907C90F002964D129209A490870002042
:1024D000984948708820974988704C209549C87061
:1024E0004B209449087145209249487156209149E2
:1024F00088714F208F49C87100208E4908720020D2
:102500008C49487200208B49887200208949C87222
:1025100000208849087300208649487300208549B7
:10252000887300208349C8730020824908743120D1
:102530008049487432207F498874FF207D49C874DF
:10254000FF207C490875FF207A4948758820794921
:10255000887577207749C87500200400132C05D2B0
:10256000FF20744909190876641CF7E700F076FA31
:10257000D1490860D0480068FFF7EEFE6C4800784B
:10258000022101436A48017000F044FFCE4908600F
:1025900059E000F0AFFA0500012D4DD164480078F4
:1025A000FD21014062480170A6484078BB2802D155
:1025B000FFF787FD47E0A34880780500882D33D1D9
:1025C000A048807D05009F48C07DFF21C94301438D
:1025D0000E00F04385421AD1280000F08EFF00283B
:1025E00012D09948007801F095F805000A276F434A
:1025F0009648007801F08EF838180600300000F098
:1026000099FF02209249087000F072FB01E000F08F
:102610005BFB8C48C3798B4882798A484179894829
:10262000007900F08AFF0EE0F32D02D1FFF749FD9B
:10263000FCE700F049FB06E0022D02D100F044FB6C
:1026400001E000F022FBF1BD04000240D0050020B3
:10265000200002402838014024000240D00400201D
:10266000280002402038014010B531480078C0B23F
:1026700040080100C907C90F00291DD105202D49B7
:10268000087000202B49487003202A49887000F008
:10269000EFFA00F0E3F98849086087480068FFF71F
:1026A0005BFE23480078022101432148017000F0BD
:1026B000B1FE854908602BE000F01CFA0400012CF3
:1026C00024D160484078BB2802D1FFF7FAFC1FE014
:1026D0005C4880780400832C0DD15A4800F06CFBD4
:1026E000002802D000F004FB01E000F0EDFA012028
:1026F000574908700CE0F92C05D1002054490870A6
:1027000000F0F6FA04E000F0DFFA01E000F0BDFAB4
:1027100010BD0000083801401C000240300002409B
:102720003400024024380140380002403C0002409E
:10273000E40700205007002010B5C6480078C0B25A
:1027400040080100C907C90F00293CD10A20C2492D
:1027500008700020C04948700620BF4988700020DA
:10276000BD49C8700020C04300F04BFE0400200E9D
:10277000B94908712000000CB7494871200AB649D0
:1027800088712000B449C8710020B3490872002044
:10279000B14948720020B04988720020AE49C87221
:1027A00000F05CF94449086043480068FFF7D4FD35
:1027B000A848007802210143A648017000F02AFED3
:1027C000414908603CE000F095F90400012C35D146
:1027D0001C484078BB2802D1FFF773FC30E0194851
:1027E00080780400862C1ED1164800F097FA002845
:1027F00002D000F07DFA01E000F066FA954800781A
:10280000C0B280080100C907C90F002903D0032006
:102810000F49087014E000F0FCFE002810D00420DE
:102820000B4908700CE0F92C05D10020084908700C
:1028300000F05EFA04E000F047FA01E000F025FA4B
:1028400010BD0000D0060020F2060020F306002094
:102850004008002010B57F480078C0B24008010051
:10286000C907C90F002931D107207B490870002012
:102870007949487052207849887000F0F9F900F0E1
:10288000DAFE040020007449C871E04372490872FE
:1028900070480078FB2101406E48017000F0DEF8BE
:1028A0000549086004480068FFF756FD694800784C
:1028B00002210143674801E0EC070020017000F0AD
:1028C000A9FD0149086043E0E807002000F012F983
:1028D0000400012C3AD11F484078BB2802D1FFF7F1
:1028E000F0FB35E01B4880780400F02C1BD1194820
:1028F000C078522814D101207D49087055480078CD
:10290000C0B280080100C907C90F002905D151488C
:102910000078F72101404F48017000F0E9F917E015
:1029200000F0D2F914E0F92C05D100F0E1F9002013
:102930006F4908700CE0862C05D100F0D9F9012010
:102940006B49087004E000F0BFF901E000F09DF968
:1029500010BD0000D006002010B53E480078C0B27F
:1029600040080100C907C90F00293CD10D203A4990
:10297000087000203849487085203749887000F079
:1029800077F900F046FE0400200E3349C87120009C
:10299000000C31490872200A2F49487220002E4944
:1029A0008872E0430400200E2B49C8722000000CFE
:1029B00029490873200A284948732000264988734A
:1029C00000F04CF8BE490860BD480068FFF7C4FC41
:1029D00020480078022101431E48017000F01AFDD2
:1029E000B849086034E000F085F80400012C2DD1CE
:1029F000C8484078BB2802D1FFF763FB28E0C548F0
:102A000080780400F02C0ED1C248C078852807D108
:102A100000F0FBFD02203649087000F069F917E06C
:102A200000F052F914E0F92C05D100F061F9002012
:102A30002F4908700CE0862C05D100F059F90120CF
:102A40002B49087004E000F03FF901E000F01DF9A7
:102A500010BD0000E40700205007002038B5012019
:102A600005000220CF49087000200400AA48007821
:102A7000401CA0421DD3A848005DC0B20009C0B2EE
:102A800000F062FEC7490222624389184870A248DA
:102A9000005D0007000F00F057FEC24902226243AA
:102AA00089188870002C02D09B48005D2D18641C8A
:102AB000DCE7E8430500EDB2280900F045FEB9491E
:102AC00002226243891848702807000F00F03CFE7C
:102AD000B44902226243891888700320B149022256
:102AE00062438918C87002204443241D200032BD6F
:102AF00040080020F0B585B000206946087100202C
:102B00000500FF2D0ADCA848405D032804D1049588
:102B10000020A549485501E06D1CF2E7FF2D00DDBE
:102B20008CE00498401E0500002D00D589E09E48E9
:102B3000405D022800D07FE0039500209A49039A67
:102B4000885404980399401A401C00900098083853
:102B500000900398401CC0B206003000401CC0B278
:102B6000029091480299415C8F48805D00F06DF8B9
:102B7000684908700098C0070DD4009840080428E0
:102B800009D3009840087D2805D200984008614983
:102B90000978884203D002206946087151E0009804
:102BA00040080090012004000398C01CC0B2060039
:102BB0003000401CC0B202907B480299415C7A48C8
:102BC000805D00F042F8534948705248407824181C
:102BD000002007000098B8421DD30398401D022131
:102BE00079434018C0B206003000401CC0B20290C9
:102BF0006D480299415C6C48805D00F026F84549BB
:102C0000C91988700098874203D24248C019807859
:102C100024187F1CDEE7E0430400E4B23D4800993D
:102C200040188078844203D002206946087102E08F
:102C300001206946087104E06D1E75E700206946B1
:102C400008716846007905B0F0BD70B505000C004C
:102C500000262800C0B200F05DFD0600360120000D
:102C6000C0B200F057FD301806003000C0B270BD91
:102C700033202949C870312027490871302026495E
:102C80004871312024498871704780B500F0C2FB3B
:102C90000C490968401AC92811D344480068401CEF
:102CA00042490860414800680B2802D3022000F026
:102CB000A1FB3F480078FD2101403D48017001BD66
:102CC000EC070020E807002080B53A480068401C67
:102CD00038490860374800680B2802D3022000F00A
:102CE00089FB33480078FD2101403148017001BD66
:102CF00080B500202F49086000202C4908602C482E
:102D00000078FD2101402A480170022000F06BFB91
:102D100001BD0000D006002050070020F8B50400D7
:102D2000E07E0500207FFF21C94301430F00F843E7
:102D3000854231D11E480078C0B2C0080100C907E1
:102D4000C90F002903D1280000F09CFC05E000F029
:102D500072FC0500280000F095FCE07800060500F4
:102D6000207900042D18607900022D18A0792D1803
:102D7000280000F0B0FC607A00060500A07A00048C
:102D80002D18E07A00022D18207B2D18280000F065
:102D9000ABFC0120060001E0002006003000C0B2BC
:102DA000F2BD0000D0040020D0050020F007002074
:102DB000E4070020F407002038B50400E07905009E
:102DC0002900207A05020D432900607A05040D438D
:102DD0002900A07A05060D43280000F01DFC012003
:102DE00032BDFEE780B500F00DF89E499E4A12689C
:102DF00012091207120F895CC8409C4908609B4861
:102E0000006802BDF8B500240020009000250026CF
:102E100000279548006804000C202040042802D0B8
:102E2000082803D01DE0924807001CE09148A10C3F
:102E30000907090F405C05008F4890490968090798
:102E4000090F405C0090E00306D58948009900F026
:102E500007FD6843060002E0894868430600370022
:102E600001E0834807003800F2BD86480068012170
:102E70000143844801607C480068834901407A48E6
:102E8000016080480068814901407E4801607D48BA
:102E900000687F4901407B480160734800687D49B4
:102EA000014071480160754800680F2188437349EB
:102EB000086079480068132188437749086077489B
:102EC00000680100C907C90F7448016000207449F7
:102ED0000860704700B56B48006872490140694856
:102EE0000160684800688001FBD4644800680F21D5
:102EF00088436249086061480068604908605A4830
:102F00000068694901405848016057480068A0219D
:102F100089030143544801605A48006880214904EC
:102F2000014358480160574800688001FBD55F485D
:102F30000068012101435D4801604B480068F021B1
:102F400088434949086048480068474908604D4837
:102F500000688001FBD5444800680321884342494A
:102F6000086041480068022101433F4801603E4833
:102F700000680C2101400829F9D13B4800684C4900
:102F800001403948016038480068374908604948BD
:102F90000068012101434748016000BD00B5C0B28F
:102FA000012807D144490968802292020A43424914
:102FB0000A6055E0C0B2022807D13F490968802263
:102FC000D2020A433C490A604AE0C0B2032807D152
:102FD00039490968802212030A4337490A603FE0F1
:102FE000C0B2042807D134490968802252030A4339
:102FF00031490A6034E0C0B2052807D12E4909687A
:103000008022D2030A432C490A6029E0C0B2062874
:1030100007D12A4909688022D2030A4327490A6056
:103020001EE0C0B2072807D1244909688022D201D6
:103030000A4322490A6013E0C0B2002806D11E49A3
:10304000096801220A431C490A6009E0C0B2082845
:1030500006D11A490968802212010A4317490A60F9
:1030600000BD00002849000804100240C8000020EC
:1030700000127A0038490008484900082C10024024
:1030800000093D00001002400CB8FF00FFFFF6FEF3
:10309000FFFFFBFFFFFFC0FF301002403410024073
:1030A00008100240FFFFFFFEFFFFC2FF00200240AA
:1030B000FFF8FFFF0C1002401410024018100240ED
:1030C00070B40468032502264E43B540AC43046047
:1030D000C4682300032402254D43AC40A3431D00D4
:1030E000D2B202244C431300A3402B43C36070BCF4
:1030F000704770B505682C00032502264E43B54085
:10310000AC432600012402254D43AC403443046007
:1031100085682C00032502264E43B540AC432600AB
:10312000DBB202254D431C00AC403443846045684B
:103130002C0001258D40AC43112A13D12500012418
:103140008C402C434460C5682C00032502264E4366
:10315000B540AC432600012402254D43AC40344326
:10316000C46008E04460C5682C00032502264E4375
:10317000B540AC43C46070BDF0B50400059DC9B254
:1031800008290EDA266A30000F2604274F43BE4076
:10319000B043070004264E432800B0403843206265
:1031A00013E0666A30000F26B4460F00083F04267D
:1031B00077436646BE40B04306000F00083F042038
:1031C00047432800B8403043606226683000032639
:1031D00002274F43BE40B0430700022002264E4361
:1031E000B04038432060A6683000032602274F43D2
:1031F000BE40B0430700DBB202264E431800B04089
:103200003843A0606668300001268E40B043122A21
:1032100013D106000120884030436060E66830002A
:10322000032602274F43BE40B04307000120022679
:103230004E43B0403843E0600EE06060E668300026
:10324000032702264E43B740B84307000120022659
:103250004E43B0403843E060F0BD10B50300D2B239
:10326000002A03D001208840986104E0012408006E
:10327000103084409C6110BD0269012088401040DC
:103280007047FEE7002202600268084B13430360A8
:103290004268074B13404360C1604268054B1340CE
:1032A000436082682A239A43826070470C80000042
:1032B000FFCFFFFFFFB7FFFF016801220A43026053
:1032C0007047FEE710B402680124A243026002685E
:1032D00013001A00094B13401A000B684C681C437A
:1032E0008B682343CC681C430B6923434C691C4304
:1032F0008B6923431343036010BC70470FC0FFFF6B
:1033000010B50400601E2849086000210020C04359
:1033100000F007F8002025490860072024490860CC
:1033200010BDF0B540B2002821D5224C40B20207B2
:10333000120F083A9508042255431E4A40B203076B
:103340001B0F083B9B0804267343D258FF238607B4
:10335000B60F08277E43B3409A438B01DBB2860742
:10336000B60F08277E43B340134363511AE0124A55
:1033700040B2830804246343D258FF238407A40F78
:1033800008256C43A3409A438B01DBB28407A40F4A
:1033900008256C43A3401343074A40B28408042520
:1033A0006C431351F0BD000014E000E018E000E0B1
:1033B00010E000E01CED00E000E400E080B500F06B
:1033C0001EFB002807D1FEF76BFF002803D100F099
:1033D0001FFB002803D0012000F00CF802E00120C0
:1033E00000F001F801BD0100094A12688A43084B48
:1033F0001A6070470100064A12680A43044B1A60BB
:10340000704701000800024A12681040704700002F
:10341000E00700202C480068704710B50020040029
:10342000302C0AD2A0002949401800688021890563
:10343000042262438850641CF2E700F079FBFFF736
:1034400049FD00F036F8FFF7CDFCFA21890000F0C5
:1034500007FA04002000FFF753FF00210020C043BB
:10346000FFF75FFF0120FFF799FD0220FFF796FDB0
:103470000520FFF793FD0323012206211448FFF7DF
:1034800038FE10BD80B500F05DFB01BD80B500F0D9
:103490006EFB01BD80B5FFF7E8FC01BD70470A482F
:1034A0000068401C08490860704700B5FEE7704797
:1034B0007047084909680800032188430100032078
:1034C00008430449086070472008002000200008D5
:1034D000001400480000014080B5002084490870B5
:1034E0000020844908600020834908600020834947
:1034F00008601020FFF77EFF01BD38B50400062CE0
:1035000005D0052C03D0072C01D0042C07D17B4813
:1035100004601020FFF767FF0120050007E010207E
:10352000FFF768FF002075490860002005002800AB
:10353000C0B232BD72490860704730B5C0B23128A0
:103540000DD1C9B234290AD1D2B2302A07D1DBB2A7
:10355000302B04D1AF24E4006A4D2C6013E0C0B2DC
:1035600031280DD1C9B230290AD1D2B2302A07D1BF
:10357000DBB2302B04D1FA24A400624D2C6002E0AF
:103580000024604D2C6030BD5E48006870475C4888
:103590000068704759480068704755480078704780
:1035A00010B50400200052490978C0B2884201D009
:1035B000FEF769FE4E48047010BD00B5C0B2002889
:1035C0000ED051490968802212060A434E490A600A
:1035D0004E490968802292010A434C490A600CE076
:1035E000494909688022D2050A4347490A60474988
:1035F0000968474A0A4045490A6000BD42480068D8
:103600000121014340480160704700203E490860A5
:1036100070473D48006870473C490860704700B5F6
:103620003A490968890402D40021080001E0012117
:103630000800C0B200BD00B52D490978012902D1AA
:10364000042108001DE02A490978022902D1082135
:10365000080016E026490978032902D12021080034
:103660000FE023490978042902D10121080008E06C
:103670001F490978052902D10221080001E0002133
:10368000080000BD00B5810703D50521184A117057
:1036900020E0C10703D50421154A11701AE0810604
:1036A00003D50321124A117014E0010703D502214A
:1036B0000F4A11700EE0C10603D502210C4A1170A9
:1036C00008E0410703D50121094A117002E00021F9
:1036D000074A117000BD0749086070470548006837
:1036E000704705480068704703490860704700004C
:1036F0004308002024080020280800202C0800206F
:103700003008002034080020380800203C08002041
:10371000FFDFFFFF00B5010000220A00D2B2302A0D
:1037200006DBD2B23A2A03DA303A1000C0B20AE01D
:10373000D2B2412A06DBD2B2472A03DA373A100066
:10374000C0B200E0002000BD0007000F0149085C86
:10375000704700005849000800B50100002901D158
:1037600020207CE0C80701D5002078E0880701D53B
:10377000012074E0480701D5022070E0080701D558
:1037800003206CE0C80601D5042068E0880601D556
:10379000052064E0480601D5062060E0080601D552
:1037A00007205CE0C80501D5082058E0880501D550
:1037B000092054E0480501D50A2050E0080501D54C
:1037C0000B204CE0C80401D50C2048E0880401D54A
:1037D0000D2044E0480401D50E2040E0080401D546
:1037E0000F203CE0C80301D5102038E0880301D544
:1037F000112034E0480301D5122030E0080301D540
:1038000013202CE0C80201D5142028E0880201D53D
:10381000152024E0480201D5162020E0080201D539
:1038200017201CE0C80101D5182018E0880101D537
:10383000192014E0480101D51A2010E0080101D533
:103840001B200CE0C80001D51C2008E0880001D531
:103850001D2004E0480001D51E2000E01F2000BD0F
:103860000022030A8B420BD203098B4219D2430870
:103870008B422ED2411A00D2014652411046704767
:10388000FF2209023FD012068B4205D31212090211
:103890008B4201D31212090203098B4219D300E0B3
:1038A000090AC3098B4201D3CB01C01A52418309D3
:1038B0008B4201D38B01C01A524143098B4201D381
:1038C0004B01C01A524103098B4201D30B01C01AAC
:1038D0005241C3088B4201D3CB00C01A5241830826
:1038E0008B4201D38B00C01A524143088B4201D353
:1038F0004B00C01A5241884200D3401A5241CFD2E5
:1039000001461046704708B5C046C04608BDFEE7F0
:1039100080B5012200218048FFF7D2FB01220A2155
:103920007D48FFF7CDFB01220B217B48FFF7C8FB49
:1039300001220D217848FFF7C3FB01220E217648B2
:10394000FFF7BEFB01220F217348FFF7B9FB0122ED
:1039500006219020C005FFF7B3FBFFF75BFD0A3897
:103960006E4908606E480078012101436C4801707F
:103970006B480078FB210140694801706848007875
:10398000FD2101406648017001BD38B564480078EA
:103990000100C907C90F002922D06248006805004C
:1039A000FFF738FD5D490968401A0A280BD3FFF775
:1039B00031FD5A49086000F034F80400200000F09E
:1039C00075F85849086057480068684056490860CB
:1039D000554800685349096888435349086005E021
:1039E0004F480078022101434D48017031BD4D49D7
:1039F0000968084070474C490968084070474848C2
:103A000000780100C9B289080800C007C00F7047DC
:103A1000434800780100C9B249080800C007C00F38
:103A2000704710B50020040000213B48FFF724FC3C
:103A3000002802D12000012404430A213648FFF760
:103A40001BFC002802D12000022404430B21324831
:103A5000FFF712FC002802D12000042404430D21AA
:103A60002D48FFF709FC002802D120000824044358
:103A70000E212948FFF700FC002802D12000102465
:103A800004430F212448FFF7F7FB002802D1200050
:103A90002024044306219020C005FFF7EDFB0028F9
:103AA00002D1200040240443200010BD70B5010065
:103AB0000B0000242200032A07D21D001B4B042404
:103AC00054431B592B43521CF5E7184CE4681C4027
:103AD00020000B0000242200032A07D21D00134BF4
:103AE000042454431B592B40521CF5E718430F4C38
:103AF000E06002242200002A0BD00C4C0425554320
:103B00006419241F2468094D04265643AC51521EE3
:103B1000F1E7064C216070BD000400480408002055
:103B2000F8070020FC07002000080020D007002034
:103B300003480068102101430148016070470000FC
:103B40000020024000B50C480C4908600C480B49A5
:103B5000086000200B4908600B480C4908600C48BD
:103B600000680028FBD10B480449086000BD0948E3
:103B70000249086070470000CCCC000000300040D3
:103B80005555000004300040FF0F00000830004091
:103B90000C300040AAAA000080B5002301220021B9
:103BA0009020C005FFF7A5FA0023012201219020F3
:103BB000C005FFF79EFA0023012202219020C005D4
:103BC000FFF797FA0023012203219020C005FFF799
:103BD00090FA0023012204219020C005FFF789FA02
:103BE0000023012205219020C005FFF782FA002260
:103BF00000219020C005FFF730FB0022012190201A
:103C0000C005FFF72AFB002202219020C005FFF724
:103C100024FB002203219020C005FFF71EFB002299
:103C200004219020C005FFF718FB002205219020F9
:103C3000C005FFF712FBFFF7EDFB7B49086000F0C2
:103C40005AFA7A480078012101437848017001BD91
:103C500077490870704780B50120FFF7D2FB002834
:103C600005D03F2000F0EAF800F045FADBE0022042
:103C7000FFF7C7FB002804D11020FFF7C2FB002884
:103C800005D03F2000F00DFA00F035FACBE068488F
:103C90000078012805D1122000F0D0F800F02BFAAE
:103CA000C1E063480078022805D10C2000F0C6F876
:103CB00000F021FAB7E05E480078032840D1FFF712
:103CC000A9FB5C490968401A5B49884208D25748F9
:103CD0000078C0B2C0080100C907C90F00291DD172
:103CE00052480078C0B2C0080100C907C90F0029B6
:103CF00006D04E480078F72101404C48017009E099
:103D000000F072F9B749086048480078082101437B
:103D100046480170FFF77EFB46490860434800783B
:103D2000C0B2C0080100C907C90F002904D0AD48BE
:103D3000006800F0B6F976E0002000F07FF872E04D
:103D40003B480078042805D10C2000F0AAF900F0C7
:103D5000D2F968E03648007805285DD1FFF75AFBB4
:103D600034490968401A344988421DD32F480078E5
:103D7000C0B2C0080100C907C90F002906D02B48EE
:103D80000078F72101402948017009E000F0E3F8CC
:103D900094490860254800780821014323480170B0
:103DA000FFF738FB2349086020480078C0B2C008FC
:103DB0000100C907C90F002928D0FFF72BFB1A49BA
:103DC0000968401AC8282ED318480078C0B24008A5
:103DD0000100C907C90F002909D0002000F02EF802
:103DE00012480078FD2101401048017009E07D482B
:103DF000006800F023F80D480078022101430B48C9
:103E00000170FFF707FB084908600CE0FFF7C5FBEE
:103E1000C0B200F070F806E0FFF7BFFBC0B200F0E0
:103E20006AF800F068F901BD0C08002008080020BD
:103E30004108002010080020B80B000010B5040055
:103E4000E00606D4002204219020C005FFF705FA01
:103E500005E0012204219020C005FFF7FEF9E007EC
:103E600006D4002200219020C005FFF7F6F905E0F6
:103E7000012200219020C005FFF7EFF9200706D4AA
:103E8000002203219020C005FFF7E7F905E0012299
:103E900003219020C005FFF7E0F9600706D4002257
:103EA00002219020C005FFF7D8F905E00122022188
:103EB0009020C005FFF7D1F9A00706D40022012108
:103EC0009020C005FFF7C9F905E0012201219020EB
:103ED000C005FFF7C2F9A00606D4002205219020F4
:103EE000C005FFF7BAF905E0012205219020C005C1
:103EF000FFF7B3F910BD10B50400E4B2002C03D1F4
:103F00000120FFF79BFF25E0E4B2022C03D104203F
:103F1000FFF794FF1EE0E4B2012C03D10820FFF765
:103F20008DFF17E0E4B2042C03D11020FFF786FFC9
:103F300010E0E4B2032C03D10220FFF77FFF09E079
:103F4000E4B2052C03D12020FFF778FF02E0012026
:103F5000FFF750FA10BD70B5FFF7C0FB0600002058
:103F60000400202C19D26B48006880210906884281
:103F700009D068480068002805D0664800684000FD
:103F80006449086002E001206249086061480068F5
:103F90003040002801D1641CE3E75E480068FFF769
:103FA000DBFB0400202C19D2FFF7F4FA062805D118
:103FB0005948042161434058050011E0FFF7EAFA2F
:103FC000052805D15548042161434058050007E004
:103FD0005348042161434058050001E000200500DA
:103FE000280070BD1408002070B5FFF7D3FA06282A
:103FF00005D1FFF776FB4B4901400E000EE0FFF7BD
:10400000C9FA052805D1FFF76CFB474901400E00AE
:1040100004E0FFF766FB434901400E000020040066
:10402000202C19D24148006880210906884209D015
:104030003E480068002805D03C48006840003B49E5
:10404000086002E0012039490860384800683040C3
:10405000002801D1641CE3E734480068FFF77CFBCB
:104060000400202C19D2FFF795FA062805D1304814
:10407000042161434058050011E0FFF78BFA052841
:1040800005D12C48042161434058050007E02A4827
:10409000042161434058050001E00020050028008C
:1040A00070BD10B50400FFF7B5F924490968401A3E
:1040B000C8281FD3FFF7AEF92049086020480078D0
:1040C000C0B240080100C907C90F002909D01C4827
:1040D0000078FD2101401A4801700020FFF7AEFE74
:1040E00008E01748007802210143154801702000BC
:1040F000FFF7A4FE10BD80B5FFF78CF911494018F9
:10410000114908600E480078082101430C480170ED
:1041100001BD0000C0000020FC450008FC4600086E
:10412000FC440008085E820408270600C400002042
:104130007C4600087C4700087C4500080C080020ED
:104140000808002048F4FFFF1008002080B5002078
:10415000BA490870FFF75EF9B9490860B9480078B4
:1041600001210143B748017001BD80B5B548007811
:104170000100C907C90F002938D0B04800780028CD
:1041800002D100F03AF837E0AC480078012802D1BB
:1041900000F012F930E0A9480078022802D100F0BE
:1041A00053F929E0A5480078032802D100F082F9EC
:1041B00022E0A2480078042802D100F088F91BE030
:1041C0009E480078052802D100F065F914E09D486A
:1041D0000078022101439B4801703F20FFF707FC54
:1041E000002809D100209549087005E0954800781D
:1041F000022101439348017001BD80B5FFF70AF920
:104200008F490860FFF76AFA002803D00520FFF7FE
:104210001FFD02E00020FFF71BFDB3480078FB21E3
:104220000140B1480170FFF7B5F9042809D1FFF743
:10423000ABF9AF21C900884203D1FFF7A8F91728CD
:1042400011D2FFF7A7F9042805D1FFF79DF9FA214C
:104250008900884207D0FFF79DF9062814D1FFF79F
:1042600096F9142810D3FFF7DAF9002806D09E48F3
:104270000078082101439C48017005E09A480078C5
:10428000F7210140984801704020FFF7B0FB00285B
:1042900006D09548007808210143934801700AE050
:1042A0004020FFF7A8FB002805D08F480078F721B1
:1042B00001408D4801701220FFF799FB122809D1A7
:1042C00001205E49087088480078FB21014086483B
:1042D000017070E00C20FFF78AFB0C2809D1022046
:1042E0005649087080480078FB2101407E480170E3
:1042F00061E00320FFF77BFB032803D103204F4934
:10430000087058E03020FFF772FB302803D10420FA
:104310004A4908704FE074480078C0B2C0080100F4
:10432000C907C90F002946D12020FFF764FB2028C8
:1043300006D10520FFF734F90020FFF789FC3AE0A9
:104340000120FFF758FB012806D10020FFF728F9CC
:104350000020FFF77DFC2EE00820FFF74CFB08282B
:1043600006D10120FFF71CF90020FFF771FC22E0C5
:104370000220FFF740FB022806D10320FFF710F9C7
:104380000020FFF765FC16E01020FFF734FB102833
:1043900006D10420FFF704F90020FFF759FC0AE0DA
:1043A0000420FFF728FB042805D10220FFF7F8F8C6
:1043B0000020FFF74DFC01BD80B51220FFF717FB71
:1043C000122836D1FFF726F81D490968401A4749D7
:1043D000884231D30120FFF73BFC1A480078C0B275
:1043E00080080100C907C90F002925D115480078A8
:1043F000C0B2C0080100C907C90F002909D111487E
:104400000078082101430F4801700120FFF7D5F81B
:1044100008E00C480078F72101400A4801700020AC
:10442000FFF7CBF8074800780421014305480170E5
:1044300002E005200149087001BD0000420800208B
:104440001C0800201808002080B50C20FFF7CFFAC8
:104450000C281CD1FEF7DEFF25490968401A2549C2
:10446000884217D30220FFF7F3FB1F480078C0B241
:1044700080080100C907C90F00290BD11A4800782C
:104480000421014318480170FFF7B8F802E0052045
:104490001949087001BD80B53F20FFF7A8FA002830
:1044A00007D13F20FFF7A7FA002802D100201249C8
:1044B000087001BD80B50320FFF7CAFB0320FFF79A
:1044C00096FA032802D005200B49087001BD80B57B
:1044D0000420FFF7BDFB3020FFF789FA302802D017
:1044E00005200549087001BD180800208813000048
:1044F0001C080020B80B000042080020010000004A
:1045000001000000040000000D0000000100000098
:104510000F0000000700000008000000020000007B
:104520000A0000000B0000000B000000110000005A
:10453000010000000E000000100000000D0000004F
:1045400012000000130000000B0000000D0000002E
:1045500016000000180000001A0000000D00000006
:104560001B0000000D0000001D0000000D000000F9
:1045700018000000020000001F0000000000000002
:1045800000000000000000003000000000000000FB
:10459000000000000000000000000000000000001B
:1045A000310000003200000034000000370000003D
:1045B00000000000350000000000000000000000C6
:1045C00038000000000000000000000000000000B3
:1045D00000000000000000003900000000000000A2
:1045E000000000003A000000000000000000000091
:1045F0000000000000000000000000000D000000AE
:104600000D000000040000000D000000010000008B
:104610000F000000070000000D0000000200000075
:104620000A0000000B0000000B0000000B0000005F
:104630000B0000000E00000010000000030000004E
:1046400012000000130000000B0000000500000035
:1046500016000000180000001A000000080000000A
:104660001B0000000D0000001D0000001E000000E7
:1046700018000000020000001F0000000000000001
:1046800000000000000000003000000000000000FA
:10469000000000000000000000000000000000001A
:1046A000310000003200000034000000370000003C
:1046B00000000000350000000000000000000000C5
:1046C00038000000000000000000000000000000B2
:1046D00000000000000000003900000000000000A1
:1046E000000000003A000000000000000000000090
:1046F00000000000000000000000000001000000B9
:1047000001000000040000000D0000000100000096
:10471000070000000A0000000B0000000B00000072
:104720000E00000010000000120000001300000046
:104730000B00000016000000180000001800000028
:104740001A0000001B000000060000000600000028
:104750000600000006000000060000000F00000038
:104760001D0000001D0000001100000002000000FC
:104770000D0000000D0000000D0000000000000012
:1047800000000000000000003000000000000000F9
:1047900000000000000000000000000031000000E8
:1047A00032000000350000000000000000000000A2
:1047B00038000000000000000000000000000000C1
:1047C000390000003A000000000000000000000076
:1047D00000000000000000000000000000000000D9
:1047E00000000000000000000000000000000000C9
:1047F00000000000000000000000000070B4012173
:10480000002213E00468001D0C4202D04D466D1ECC
:1048100064192260241D1B1F042BFAD225009E0759
:1048200001D52280AD1C0B4000D02A700368001D0A
:10483000002BE7D170BC704780B5FEF7EEFDFEF7A8
:104840004BFEFDF748FCFFF763F8FFF7A5F9FFF70C
:104850007DFCFEF717FEFEF719FEFFF796F8FFF74F
:1048600084FCFDF7C3FCFFF7F6F9FEF7A7FDF2E7BE
:1048700030B401210268001D002A0FD00368C3185C
:10488000446808300C4202D04D466D1E64191D6804
:1048900025601B1D241D121FECD0F8E730BC7047AB
:1048A00010B5074979441831064C7C44163404E0AD
:1048B000081D0A68891888470100A142F8D110BD77
:1048C000080000002800000035FFFFFF740300000F
:1048D000D00400200000000099FFFFFF0C00000042
:1048E000A4000000C0000020000000000120C0461D
:1048F000002801D0FFF7D4FF002000BF00BFFFF762
:104900009BFF00F000F880B500F002F801BDFEE763
:104910000746384600F002F8FBE7FEE720210903CE
:1049200026311820ABBEF9E70000000001020304A5
:104930000102030406070809020304050607080923
:104940000A0B0C0D0E0F10100102030405060708D8
:10495000090A0B0C0D0E0F10303132333435363757
:1049600038394142434445460148804701480047A1
:10497000953400087949000800BF00BF00BF00BFA0
:10498000FFF7B4FF010000000100000000127A00F0
:10499000FEE7FEE7FEE7FEE7FEE7FEE7FEE7FEE7EF
:1049A000FEE7FEE7FEE7FEE7FEE7FEE7FEE7FEE7DF
:0449B000FEE7FEE739
:04000005080049792D
:00000001FF
